:103E120000010C01010402011E030A96040132058D
:103E2200020206006407010108000009015A0E019E
:103E3200010F000112006413010114013C1501FA83
:103E42001664FA17FFFF1D0007200007240002274F
:103E520001012F013C30010132010335FFFF36031E
:103E6200073CFFFF3DFFFF180002191E461A000221
:103E72001B00022D32C82E0001FAFAFA18000019AE
:103E8200FFFF1A00001B00002D32C82E0001FAFAB3
:103E9200FA18000019FFFF1A00001B00002DFFFF97
:063EA2002EFFFFFAFAFA00
:10004800900786E0FEA3E0FF7457BE0010D39F40E0
:100058000C903E1212001EE493F599804C90001407
:10006800E0D394044014900786E0FEA3E0FF903E9E
:100078001212001EE493F599802F900014E0D39497
:10008800034014900786E0FEA3E0FF903E2712008D
:100098001EE493F5998012900786E0FEA3E0FF9096
:1000A8003E3C12001EE493F59990078612000E90CC
:1000B8000786E0FEA3E0FF746C6F4E7003751300B3
:1000C80022900072E0B402087401900072F0D20C21
:1000D80090013AE090002AF090013BE090002BF06C
:1000E80090013CE090002CF0A20AB3401690013A2F
:1000F800E0700C90013BE0700690013CE0600280EB
:1001080002C20A90013AE0B4300F90013BE0B447D4
:100118000890013CE0643B60028004D20B8002C27C
:100128000BE558B40102800302024B900057E0F53A
:1001380066900062E0F568900063E0F569900074ED
:10014800E0F56A90007AE0900029F090007CE0F5F4
:100158006590007DE0F567900080E0F5649000818F
:10016800E0F563900090E0900041F0900091E090FD
:100178000042F0900092E0900043F0900093E090ED
:100188000044F0900094E0900045F0900095E090D5
:100198000046F0900096E0900047F0900097E090BD
:1001A8000048F0900099E0900033F090009AE090B9
:1001B8000034F090009BE0900035F090009CE090B7
:1001C8000036F0900079E0B4011790000A740FF03F
:1001D800A374FFF090000CE4F0A3F074029000798F
:1001E800F0900079E0B4035990000CE0FEA3E0FF22
:1001F80090000AE0FCA3E0FD1200037410123F27F0
:100208007408123F19EF900026F0EF700674FF9003
:100218000026F07400900079F090000BE090002721
:10022800F090000AE0900028F0900026E0900789FE
:10023800F0900027E090078AF0900028E090078B64
:10024800F0803F900081E07006755801756300A248
:100258000AB3402E90013AE090002AF090013BE06A
:1002680090002BF090013CE090002CF090002AE0E8
:10027800700C90002BE0700690002CE06002800269
:10028800C20AE5667003756602E568700375680260
:100298007E887F75E5668E048F05FF123F098C39CD
:1002A8008D3AE56975F0FAA4FFAEF0E5688E048F23
:1002B80005FF123F098C3D8D3E90004FE0F56090A0
:1002C800004DE0FE900069E0B5061890004CE0FE95
:1002D800900068E0B5060C90004BE0FE900059E0F5
:1002E8006E606F900069E07006900068E0600674C8
:1002F80000900059F0900069E0B402089000497439
:1003080001F08005900049E4F0900068E0B402082C
:1003180090004A7401F0800590004AE4F09000686B
:10032800E0600690004AE060028005756003800383
:10033800756004E559B55802D20C900068E0900049
:100348004CF0900069E090004DF0900059E090006A
:100358004BF0740090009EF0740090009FF07400C1
:100368009000A0F074009000A1F074009000A2F03A
:1003780074009000A3F074009000A4F07400900042
:10038800A5F074009000A6F074009000A7F0740027
:100398009000A8F074009000A9F074009000AAF0F2
:1003A80074009000ABF074009000ACF07400900002
:1003B800ADF074009000AEF074009000AFF07400DF
:1003C8009000B0F074009000B1F074009000B2F0AA
:1003D8007400900362F07401900363F0740090035A
:1003E80064F07400900365F07400900366F0740084
:1003F800900367F07400900368F074019003A2F012
:1004080074019003A3F074009003A4F074009003A7
:10041800A5F074009003A6F074009003A7F0740090
:100428009003A8F074019003E2F074009003E3F0E5
:1004380074009003E4F074009003E5F074009003F6
:10044800E6F074009003E7F074009003E8F074009D
:10045800900422F07400900423F07400900424F0B7
:100468007400900425F07400900426F07400900441
:1004780027F07400900428F022E5B554F7F5B5E5A7
:10048800B554FDF5B5C292C287C290C207E5B5540E
:10049800FBF5B5755104E55104F55290004FE0F5B0
:1004A80060900025E4F0C209E5B554FEF5B5C28EAA
:1004B800758D00758B00754C00752600752500D26A
:1004C8008E22750A00750900AE09AF0A7457BE007E
:1004D800039F5003020587903E1212001EE493907A
:1004E800004E123F3F0FBF00010EE0FC903E12127B
:1004F800001EECFEE493FFEEC39F5026AE09AF0A40
:100508000FBF00010E903E1212001EAE09AF0AE4A2
:1005180093FC903E1212001EE49390004E123F3F4F
:10052800ECF0AE09AF0A903E1212001EE493900060
:100538004E123F3FE0FC903E1412001EECFCE49388
:10054800FDECD39D4019903E1412001EE493FC90DC
:100558003E1212001EE49390004E123F3FECF0AEA4
:1005680009AF0A74022FFF50010E8E098F0A780A0C
:10057800740126F6500418E436F640030204D0222B
:10058800750A00750900AE09AF0A7415BE00039F0D
:100598005003020655903E6912001EE49390004EE7
:1005A800123F3F0FBF00010EE0FC903E6912001E93
:1005B800ECFEE493FFEEC39F5026AE09AF0A0FBFCF
:1005C80000010E903E6912001EAE09AF0AE493FCCA
:1005D800903E6912001EE49390004E123F3FECF0EB
:1005E800AE09AF0A903E6912001EE49390004E12C5
:1005F8003F3FE0FC903E6B12001EECFCE493FDECE8
:10060800D39D4019903E6B12001EE493FC903E6906
:1006180012001EE49390004E123F3FECF0AE09AF7B
:100628000A740F6F4E7006750A15750900AE09AF8A
:100638000A74022FFF50010E8E098F0A780A74017E
:1006480026F6500418E436F6400302058E22750A91
:1006580000750900AE09AF0A7415BE00039F500368
:10066800020723903E7E12001EE49390004E123F34
:100678003F0FBF00010EE0FC903E7E12001EECFE14
:10068800E493FFEEC39F5026AE09AF0A0FBF0001E7
:100698000E903E7E12001EAE09AF0AE493FC903E17
:1006A8007E12001EE49390004E123F3FECF0AE091C
:1006B800AF0A903E7E12001EE49390004E123F3F18
:1006C800E0FC903E8012001EECFCE493FDECD39D10
:1006D8004019903E8012001EE493FC903E7E12006A
:1006E8001EE49390004E123F3FECF0AE09AF0A743F
:1006F8000F6F4E7006750A15750900AE09AF0A74BA
:10070800022FFF50010E8E098F0A780A740126F60F
:10071800500418E436F6400302065C22750A007598
:100728000900AE09AF0A7415BE00039F5003020703
:10073800F1903E9312001EE49390004E123F3F0F3B
:10074800BF00010EE0FC903E9312001EECFEE49305
:10075800FFEEC39F5026AE09AF0A0FBF00010E90EF
:100768003E9312001EAE09AF0AE493FC903E93122A
:10077800001EE49390004E123F3FECF0AE09AF0A22
:10078800903E9312001EE49390004E123F3FE0FC0F
:10079800903E9512001EECFCE493FDECD39D4019AD
:1007A800903E9512001EE493FC903E9312001EE4C6
:1007B8009390004E123F3FECF0AE09AF0A740F6FF2
:1007C8004E7006750A15750900AE09AF0A74022F36
:1007D800FF50010E8E098F0A780A740126F650041C
:1007E80018E436F6400302072A22054D22054C225A
:1007F800054EC2CF2290F800E4936406600280FEA2
:1008080075840175A70075FF80900788E4F075C9A5
:100818001075A70F75A1C775A70075D90075CEFF0C
:1008280075A70F75F1FE75F2FF75F33775F47875D6
:10083800A4BA75A5FF75A60775AE0075AFFF75D488
:100848008175D5FF75D6FF75D7FFC293C294C29143
:10085800E5B554BFF5B5E5B554DFF5B5E5B554EFE5
:10086800F5B5E5B5547FF5B5E5B554F7F5B5E5B596
:1008780054FDF5B575A70075A20175A14775F8096E
:1008880075BC0175BE0475BD6C75BE0775BDA075D8
:10089800BE0875BD0175BC0075BB1875BC2075BA5E
:1008A8000875E88075D11375A70F75E10575E20025
:1008B80075C740759700759780740A123EF9759749
:1008C800C0E5975420700280F8758F0275A700D292
:1008D800AF75980075A90C75A70F75AB4375ADFB7F
:1008E80075AC1E75A700758911758E00758C00751D
:1008F8008A00D2A9D28C758D00758B00D2ABD28EAE
:1009080075CD0075CC0075CA0075CB00D2ADC2CFCD
:10091800D2CA7591047592007593CD75EF0675D995
:100928004075CF01900786E4F0A3F07513007514A5
:1009380000C299D20AC20D12048174C8F51875173D
:100948000012266075A70FE5FB90001AF0E5FA90F3
:10095800001BF0E5F990001CF075A70090F800E482
:1009680093F508122797122CD1900789E09000265A
:10097800F090078AE0900027F090078BE09000281D
:10098800F090078CE0900029F090078DE0F56690D4
:10099800078EE0F56890078FE0F569900790E0F51D
:1009A8006A900791E0F565900792E0F567900793E4
:1009B800E0F564900794E0F563900795E090002ACD
:1009C800F0900796E090002BF0900797E090002CAD
:1009D800F0900798E0900041F0900799E09000426D
:1009E800F090079AE0900043F090079BE090004455
:1009F800F090079CE0900045F090079DE09000463D
:100A0800F090079EE0900047F090079FE090004824
:100A1800F09007A0E0900033F09007A1E090003438
:100A2800F09007A2E0900035F09007A3E090003620
:100A3800F07400900082F090013AE0700C90013B55
:100A4800E0700690013CE060028004C20A8002D295
:100A58000A90F807E493900021F0900021E0440AFE
:100A6800900021F0900021E054FE900021F07406DF
:100A7800900012F07402900013F090F802E4939042
:100A88000014F07403900015F07403900016F074CD
:100A98001B900017F07405900018F0900014E0B453
:100AA80004067404900018F0900014E0B40306746F
:100AB80003900018F07405900019F090F804E4937E
:100AC80090001DF0740090001EF090F805E49390DB
:100AD800001FF090F806E493900020F074FF900057
:100AE80022F0745A900125F07446900126F0742083
:100AF800900127F07434900128F07448900129F08F
:100B0800745090012AF0743290012BF074349001E3
:100B18002CF0742090012DF0743490012EF0742D77
:100B280090012FF07453900130F0746F900131F000
:100B3800746C900132F07420900133F090007AE0E8
:100B4800D394014006740090007AF07558017559E5
:100B580001740390004CF01200C91204CA900014EA
:100B6800E0B404051206568011900014E0D39404F2
:100B78004005120588800312072412268CE5B55417
:100B8800FEF5B5900025E4F0900786E4F0A3F07533
:100B98002400752300754800752A007529007549D9
:100BA80000753200753100754A007554007555009E
:100BB800755A0075510475520175343C75330075CA
:100BC8007000756F007571CD7556007557007543C7
:100BD80000754400754500754600755B0075470053
:100BE800754200754100900006E4F0A3F0900008FB
:100BF800E4F0A3F0755E00755F0090000E74FDF0E0
:100C0800A374E8F0900023E4F07464900024F0C228
:100C180000D201C202D203754D00756D00C297C2A1
:100C2800A0C296C295C2A2C20C7E017F0090002885
:100C3800E0123F27900027E02FFF50010E90000A96
:100C4800EEF0A3EFF0900026E0700674FF90002607
:100C5800F090000AE0FEA3E0FFEFD394FFEE940FBC
:100C6800400790000AE4F0A3F07400900071F0745B
:100C780000900079F07400900082F0740090008D6C
:100C8800F074009000B4F0E5677003756704743A77
:100C980090074EF074FD90074FF09003D4E0900455
:100CA80014F0D2B0D2B7D2A7D2A6D2B1D2A3C2077B
:100CB800A2B6B39204A2B3B39205D29CD2EC75CF7C
:100CC80001A298B34005C298123035E5136006A218
:100CD80099B3B340028005C2991235A5E5146401A1
:100CE8006005E514B4040280D5E54DD39405400CA5
:100CF800E55AC394C85002055A754D00E571C3946E
:100D0800F0501A786F12003FAE6FAF70EFD394E8CF
:100D1800EE940340080571757000756F00C28E7EF1
:100D2800047F00E54C123F27E58D75F004A4FDAC67
:100D3800F0EF2DFDEE3CFCE58B75F04084FF7E0066
:100D4800ED2FFFEC3EFE8E258F26D28EA2B6300404
:100D580001B35003020E99A2B6300401B350030246
:100D68000E99A2B640670554A20D400575FFA0D2A2
:100D78000DE5B54401F5B5900024E4F0E554D395AC
:100D88006640487C887D75AE25AF26123D318E239E
:100D98008F24E5482FFF50010E7401123F198E234E
:100DA8008F24852448755401C28E758D00758B007B
:100DB800754C00D28E7403BE00039F500690002528
:100DC8007401F0E543B40603754300D204A2B6B338
:100DD8005003020E99C20490006BE060181236E6C8
:100DE800A200B34008E5B54408F5B58006E5B5545A
:100DF800F7F5B58002C20090006EE0601812383B2B
:100E0800A202B34008E5B54402F5B58006E5B5543D
:100E1800FDF5B58006E5B554FDF5B5A207B3400468
:100E2800D2968002C296900059E06004D295800262
:100E3800C29590004AE0B40104D2978002C297900C
:100E48000049E0B40104D2A08002C2A0A209B340C4
:100E580004D2A28002C2A2900018E0FE900014E022
:100E6800C39E4009900014E0D39408400974FB9095
:100E78000023F012048190001DE0601590001DE031
:100E8800FE900017E06E600974FE900023F01204D3
:100E980081C2CA7E017F00E54E123F27E5CD2FFFB4
:100EA80050010E8E278F28D2CAE565B401489000FC
:100EB8000EE0FCA3E0FDEFC39DEE9C4039B208E5CF
:100EC8002A45296013A208B34008E5B54404F5B5DE
:100ED8008006E5B554FBF5B590000EE0FEA3E0FFF3
:100EE800900010E0FCA3E0FDEF2DFDEE3CFC90002F
:100EF8000EECF0A3EDF0A2B3300501B35003020FDE
:100F0800E7A2B3300501B35003020FE7A2B35003C1
:100F1800020FE00555A20D400575FFA0D20DE5B5FD
:100F28004401F5B5900024E4F0E555D395685003E5
:100F3800020FDE7CEA7D60AE27AF28123D318E2994
:100F48008F2AE569123F2774FF8E048F05FF123F31
:100F5800098C298D2AE5492DFD50010C74018C0658
:100F68008D07123F198E298F2A852A49A209B34075
:100F7800157464123F27900067E08E048F05FF12F6
:100F88003F098C298D2A75550190000EE0FEA3E0DB
:100F9800FFAC27AD2812000390000EEEF0A3EFF08F
:100FA800E567FF123F09740AFF123F0990007BE0D2
:100FB8008C068D07123F2774148E048F05FF123F8D
:100FC80009900010ECF0A3EDF0C2CA75CD0075CC05
:100FD80000754E00D2CAD205A2B3B34002C2059032
:100FE8000025E0B40107E556C3940640030215F353
:100FF800E56D90263FF8282873900059E0C39402C5
:101008004003021155E551D394015003021155E5EF
:101018005175F040A4FFAEF090031212001EE0C319
:1010280095455018E55175F040A4FFAEF0900311B6
:1010380012001EE0F52E752D00021155E55175F0D0
:1010480040A4FFAEF090031012001EE0C395454087
:10105800030210F1E55175F040A4FFAEF0900311C2
:1010680012001EE55175F040A4FFAEF0E0FC9003BD
:101078000F12001EECFEE0FFEEC39FFEE5518E044A
:1010880075F040A4FFAEF090031012001EE0F404C7
:1010980025458C0088F0A4FFAEF0E5518F048E053D
:1010A80075F040A4FFAEF090031212001EE55175D2
:1010B800F040A4FFAEF0E0FA90031012001EEAFE22
:1010C800E0FFEEC39FFECDCCCD8E07123F09E55160
:1010D80075F040A4FFAEF090030F12001EE02DFD46
:1010E80050010C8C2D8D2E8064E55175F040A4FFC5
:1010F800AEF090030F12001EE55175F040A4FFAE4C
:10110800F0E0FC90030E12001EECFEE0FFEEC39F21
:101118008545F0A4FFAEF0E5518F048E0575F040CB
:10112800A4FFAEF090031012001EE0FECDCCCD8ED1
:1011380007123F09E55175F040A4FFAEF090030E89
:1011480012001EE02DFD50010C8C2D8D2E756D01A9
:101158000215F3900059E0C394024003021308906B
:10116800004FE0D3955150030212B1E55175F0409C
:10117800A4FFAEF090031812001EE0C39545501866
:10118800E55175F040A4FFAEF090031712001EE081
:10119800F52C752B000212B1E55175F040A4FFAE95
:1011A800F090031612001EE0C39545400302124D4D
:1011B800E55175F040A4FFAEF090031712001EE54C
:1011C8005175F040A4FFAEF0E0FC90031512001E2C
:1011D800ECFEE0FFEEC39FFEE5518E0475F040A4DF
:1011E800FFAEF090031612001EE0F40425458C00B3
:1011F80088F0A4FFAEF0E5518F048E0575F040A489
:10120800FFAEF090031812001EE55175F040A4FFE0
:10121800AEF0E0FA90031612001EEAFEE0FFEEC3FD
:101228009FFECDCCCD8E07123F09E55175F040A445
:10123800FFAEF090031512001EE02DFD50010C8C3E
:101248002B8D2C8064E55175F040A4FFAEF090031F
:101258001512001EE55175F040A4FFAEF0E0FC90B9
:10126800031412001EECFEE0FFEEC39F8545F0A4B8
:10127800FFAEF0E5518F048E0575F040A4FFAEF087
:1012880090031612001EE0FECDCCCD8E07123F094A
:10129800E55175F040A4FFAEF090031412001EE073
:1012A8002DFD50010C8C2B8D2CE551B40122E560ED
:1012B800D39401401BE551C395565014E545C3949A
:1012C80005500D90035FE0A829B80006952A400252
:1012D8008003755102E551B5602290004FE0D39527
:1012E800514019E55175F040A4FFAEF09003171274
:1012F800001EE0A823B8000695244002800205607D
:10130800756D020215F3900059E0B4022AE5517593
:10131800F040A4FFAEF090031712001EE0F52C7504
:101328002B00E55175F040A4FFAEF090030E1200BB
:101338001EE0F52E752D00900059E0B4030F9000C3
:1013480051E0F52C752B00752E00752D00756D0379
:101358000215F3E55175F040A4FFAEF0900320129A
:10136800001EE0C3955A400302142A900049E07019
:1013780036E551D394014029AE23AF24AC2DAD2ED0
:10138800EDD39FEC9E401AE55175F040A4FFAEF0F6
:1013980090031E12001EE0A829B80005D3952A5014
:1013A80002800215518034E551D394024029AE23BE
:1013B800AF24AC2DAD2EEDD39FEC9E401AE55175B0
:1013C800F040A4FFAEF090031E12001EE0A829B85A
:1013D8000005D3952A500280021551E551C3956046
:1013E800502FE551C395565028AE23AF24AC2BADF2
:1013F8002CEFD39DEE9C4019E55175F040A4FFAE4B
:10140800F090031F12001EE0A829B80006952A4094
:101418000280020551C290E55165526005C2077508
:101428005A00756D040215F3E55175F040A4FFAE3E
:10143800F090031A12001EE0B40117E55175F04050
:10144800A4FFAEF090032012001EE0240AC3955AB0
:101458004003021500753064752F00A207B3500BC6
:10146800900060E02405C395454003021500E5514E
:1014780075F040A4FFAEF090031D12001EE0C39566
:10148800454064E55175F040A4FFAEF090031C128E
:10149800001EE55175F040A4FFAEF0E0FC90031B80
:1014A80012001EECFEE0FFEEC39F8545F0A4FFAEE0
:1014B800F0E5518F048E0575F040A4FFAEF090035F
:1014C8001D12001EE0FECDCCCD8E07123F09E5515E
:1014D80075F040A4FFAEF090031B12001EE02DFD36
:1014E80050010C8C2F8D30AE23AF24AC2FAD30EFD4
:1014F800D39DEE9C4002D207756D050215F3E551A8
:10150800B40109900059E0C3940240030215D39036
:101518000358E0D3954550030215D3900356E0C312
:1015280095455040900357E0FE900355E0F4042E93
:10153800FE900356E0F40425458E0088F0A4FFAE23
:10154800F0900358E0FC900356E0F4042C8E048FCE
:1015580005FF123F09900355E02DFD50010C8C2B1F
:101568008D2C802C900355E0FE900354E0F4042E5B
:101578008545F0A4FFAEF0900356E08E048F05FF7A
:10158800123F09900354E02DFD50010C8C2B8D2C3B
:10159800E551C39560502FE551C395565028AE23A9
:1015A800AF24AC2BAD2CEFD39DEE9C4019E55175C3
:1015B800F040A4FFAEF090031F12001EE0A829B867
:1015C8000006952A40028003755102900049E0B454
:1015D8000106E551640160028003755102E5516519
:0B15E800526005C207755A00756D00C7
:10263F0002100102115B02130E02135B021430022F
:02264F0015066E
:1015F300900050E02402A823B80007D395244002AA
:10160300C207900025E0B40109900059E0C3940398
:101613004003021779900049E060030216C9E551BF
:10162300D394014034E55175F040A4FFAEF090032C
:101633001412001EE0A823B8001FD39524401AE516
:101643005175F040A4FFAEF090031F12001EE0A8F6
:1016530029B80005D3952A500280021551E551D3CC
:101663009401402FE55175F040A4FFAEF0900312B2
:1016730012001EE0C39545501AE55175F040A4FFD2
:10168300AEF090031E12001EE0A829B80005D39502
:101693002A500280021551E551D394014021E551AE
:1016A300D39556401AE55175F040A4FFAEF0900370
:1016B3001E12001EE0A829B80005D3952A50028007
:1016C30002155102176EE551D394024034E551756A
:1016D300F040A4FFAEF090031412001EE0A823B85C
:1016E300001FD39524401AE55175F040A4FFAEF0D6
:1016F30090031F12001EE0A829B80005D3952A50B5
:101703000280021551E551D39402402FE55175F043
:1017130040A4FFAEF090031212001EE0C3954550A3
:101723001AE55175F040A4FFAEF090031E12001E9F
:10173300E0A829B80005D3952A500280021551E587
:1017430051D394024021E551D39556401AE5517582
:10175300F040A4FFAEF090031E12001EE0A829B8CB
:101763000005D3952A500280021551E55165526058
:1017730005C207755A00900060E0D3954550099063
:101783000054E0C395455002C207900059E070032E
:101793000219DCA2A5B34008A2A4B340030219C5F1
:1017A300AE35AF367441D39F749C9E400578351295
:1017B300003FAE35AF36EFB48806EEB413028003B4
:1017C3000219A2A2A55003021865900059E0B401C2
:1017D3000B90004FE0D3956040020560900059E004
:1017E300B40253E55175F040A4FFAEF0900320120C
:1017F300001EE0C3955A503E90004FE0D3955140F0
:1018030020E551C395565019E55175F040A4FFAE3C
:10181300F090031412001EE0A823B800069524409C
:10182300028002055190004FE0F560E5516552607A
:1018330005C207755A00900059E0B4032590004F84
:10184300E0D395514007E551C39556400280020508
:101853005190004FE0F560E55165526005C2077590
:101863005A00A2A450030219A2900059E0B4016ED9
:10187300900049E07035E551D394014029E5517555
:10188300F040A4FFAEF090031E12001EE0A829B89A
:10189300000FD3952A400A1551755A00855160806F
:1018A3000385516080037560018033E551D3940251
:1018B3004029E55175F040A4FFAEF090031E1200DD
:1018C3001EE0A829B8000FD3952A400A1551755A6E
:1018D300008551608003855160800375600290002C
:1018E30059E0D394015003021996E55175F040A4D1
:1018F300FFAEF090032012001EE0C3955A4003028E
:101903001996900049E07041E551D394014034E5C4
:101913005175F040A4FFAEF090031112001EE0A831
:1019230023B8001FD39524401AE55175F040A4FF56
:10193300AEF090031E12001EE0A829B80005D3954F
:101943002A500280021551803FE551D3940240345E
:10195300E55175F040A4FFAEF090031112001EE0B4
:10196300A823B8001FD39524401AE55175F040A46D
:10197300FFAEF090031E12001EE0A829B80005D3A5
:10198300952A500280021551E55165526005C20740
:10199300755A00E556B40704055E8003755E00E5DD
:1019A30063B4010EAE35AF36EF64407005EE649C50
:1019B3006002800EA2A54003755801A2A4400375DE
:1019C3005802A2A5B3B35006A2A4B3B34002800643
:1019D300753600753500021ACAA2A5B34008A2A441
:1019E300B34003021AB6AE35AF367441D39F749C2D
:1019F3009E4005783512003FAE35AF36EFB488060A
:101A0300EEB413028003021AB6A2A5406F900068D9
:101A1300E0605A90004AE0B4010790004AE4F08085
:101A23000690004A7401F090004AE0700575600367
:101A3300800375600490004AE0B40104D2978002E9
:101A4300C297E551B4041AE55175F040A4FFAEF016
:101A530090031E12001EE0A829B80005D3952A5052
:101A6300028008755103C207755A0080037560042C
:101A7300E556B40704055E8003755E00A2A44033F7
:101A8300900069E06021900049E0B40107900049AB
:101A9300E4F080069000497401F0900049E0B4013D
:101AA30004D2A08002C2A0E556B40704055E8003F9
:101AB300755E00A2A5B3B35006A2A4B3B3400280DF
:101AC30006753600753500E5586559600690008245
:101AD300E06003021C52C29C751400751300C2CA55
:101AE300E558902651F82828738012122CD1800DC6
:0D1AF300122DAA8008122E838003122F5C92
:0F265100021AEC021AEE021AF3021AF8021AFD2C
:101B0000900029E090007AF0E566900057F0E568D3
:101B1000900062F0E569900063F0E56A900074F06F
:101B2000E56590007CF0E56790007DF0E56490004D
:101B300080F0E563900081F090002AE090013AF097
:101B400090002BE090013BF090002CE090013CF0E5
:101B5000900041E0900090F0900042E0900091F001
:101B6000900043E0900092F0900044E0900093F0E9
:101B7000900045E0900094F0900046E0900095F0D1
:101B8000900047E0900096F0900048E0900097F0B9
:101B9000900033E0900099F0900034E090009AF0CB
:101BA000900035E090009BF0900036E090009CF0B3
:101BB0007400900082F0745A900125F074469001F0
:101BC00026F07420900127F07434900128F07448B6
:101BD000900129F0745090012AF0743290012BF09A
:101BE000743490012CF0742090012DF07434900125
:101BF0002EF0742D90012FF07453900130F0746F1B
:101C0000900131F0746C900132F07420900133F047
:101C10009003D4E0900414F0743A90074EF074FDF1
:101C200090074FF01200C9900004E4F0A3F0900078
:101C3000067475F0A37430F09000087475F0A37406
:101C400030F0855859D2CA754C00D29C741B900054
:101C500023F0E556C394065005E551B55202804E77
:101C6000C207E55175F040A4FFAEF09003221200C8
:101C70001EE030E003D38001C39293E55175F0403C
:101C8000A4FFAEF090032312001EE030E003D380E7
:101C900001C39294855152AE29AF2A7405BE000348
:101CA0009F5007E545D3940550028002D290E55637
:101CB000D394055003021D73C207E551D39401402C
:101CC00059E55175F040A4FFAEF090031E12001EBE
:101CD000E0A829B80007D3952A40021551E55165BF
:101CE000526035E55175F040A4FFAEF0900322122A
:101CF000001EE030E003D38001C39293E55175F0FC
:101D000040A4FFAEF090032312001EE030E003D3A6
:101D10008001C392948551528059E556B4061A90B9
:101D200000ACE030E003D38001C392939000ADE0BB
:101D300030E003D38001C39294E556B40716AE2970
:101D4000AF2A7404BE00039F5006C293D29480044D
:101D5000D293C294E556B4081A90009EE030E00396
:101D6000D38001C3929390009FE030E003D38001C1
:101D7000C39294900072E06058E54575F00284FFCC
:101D80007E0090014E12001EE0F55CE54775F00AFA
:101D900084FF7E0090024E12001EE0F55DE55C259A
:101DA0005DD39464400BE55C255DC39464F55C8071
:101DB00003755C00E55C75F00284FF7E008F5CEFCC
:101DC000C394335007EF24CDF55C8003755CFF802E
:101DD0001CE54575F00284FF7E0090014E12001E46
:101DE000E075F00284FF7E00EF24CDF55CE595C33D
:101DF000955C4004C2928002D292A207B34005E5EE
:101E000056B407037571CDE595C395714004C2873B
:101E10008002D287E543C394064003022417A2ED53
:101E2000B35003022417C2EDE5436003021F797E1D
:101E3000017F00E5BE123F27E5BD2FFF50010E9048
:101E40000000EEF0A3EFF0900029E0B401177E0F40
:101E50007FFF900000E0FCA3E0FD12000390000073
:101E6000EEF0A3EFF0900079E0B4025B900000E0A8
:101E7000FEA3E0FF90000AE0FCA3E0FDEDD39FECA1
:101E80009E400F900000E0F8A3E090000AC8F0A385
:101E9000C8F0900000E0FEA3E0FF90000CE0FCA37F
:101EA000E0FDEFD39DEE9C400F900000E0F8A3E032
:101EB00090000CC8F0A3C8F0900000E0FEA3E0FF83
:101EC0007404123F198F44900079E0706090000014
:101ED000E0FEA3E0FF90000AE0FCA3E0FDEFD39D4D
:101EE000EE9C400D120003900000EEF0A3EFF08096
:101EF00007900000E4F0A3F0900000E0FEA3E0FFF4
:101F00007410123F27900026E08E048F05FF123FC9
:101F100009900000ECF0A3EDF07400D39D74019CD7
:101F20004008900001E0F54480037544FFE54475E6
:101F3000F00AA4FFAEF074198E048F05FF123F095A
:101F40008D45ED2532FFAE3150010E7401123F195F
:101F50008F45854532753100EFD394624003754556
:101F600062900072E064016006900066E0600280AA
:101F700005754301800375BB17E543B40102800377
:101F80000220697E017F00E5BE123F27E5BD2FFFDD
:101F900050010E900000EEF0A3EFF0900072E0B45C
:101FA000017EE53445336025AC33AD341DBDFF0102
:101FB0001C8F028E038C068D07903A5D12002EE472
:101FC00093FE740193FFEFC39AEE9B400280057865
:101FD00033123F51AE33AF3474B3BE0025D39F40AC
:101FE00021900000E0FCA3E0FD0FBF00010E903A3D
:101FF0005D12002EE493FE740193FFEDC39FEC9EEF
:1020000040028005783312003FAE33AF34E56A12E8
:102010003F2774648E048F05FF123F098D4780337C
:10202000900066E0602D900000E0FEA3E0FFEFD39B
:102030009400EE9408400F900066E0B40104C209D9
:102040008002D209800D900066E0B40104D20980BC
:1020500002C209900072E064026006900066E060CF
:102060000575BB168003754302E543B40202800385
:102070000221577E017F00E5BE123F27E5BD2FFFFD
:1020800050010E900000EEF0A3EFF0900072E0B46B
:10209000027EE53445336025AC33AD341DBDFF0110
:1020A0001C8F028E038C068D07903BC712002EE416
:1020B00093FE740193FFEFC39AEE9B400280057874
:1020C00033123F51AE33AF3474B3BE0025D39F40BB
:1020D00021900000E0FCA3E0FD0FBF00010E903B4B
:1020E000C712002EE493FE740193FFEDC39FEC9E94
:1020F00040028005783312003FAE33AF34E56A12F8
:102100003F2774648E048F05FF123F098D4780338B
:10211000900066E0602D900000E0FEA3E0FFEFD3AA
:102120009400EE9408400F900066E0B40104C209E8
:102130008002D209800D900066E0B40104D20980CB
:1021400002C209900072E07003754700900066E0DB
:102150007002C20975BB1FE543B403457E017F00D1
:10216000E5BE123F27E5BD2FFF50010E900000EEA7
:10217000F0A3EFF07409123F2774E68E048F05FF79
:10218000123F098C418D42E54A2DFD50010C74012E
:102190008C068D07123F198E418F4285424A75BBCE
:1021A00019E543B4040280030222FF7E017F00E5AB
:1021B000BE123F27E5BD2FFF50010E900000EEF04C
:1021C000A3EFF07404123F198F4BE564B401028051
:1021D0000302228C756B00756B00E56BD39407408E
:1021E00003022279E56B900041123F3FE0D3954B0B
:1021F000501AE56B900041123F3FE0F404254BFE7E
:10220000E56B900037123F3FEEF08017E56B9000D2
:1022100041123F3FE0C3954BFEE56B900037123F04
:102220003FEEF0E56BC394044009900084E0C39551
:102230006B503BE56B6029E56B900037123F3FFE2A
:10224000E0FFEE90003FE0D39F4013E56B90003736
:10225000123F3FE090003FF0E56B900040F0800EB1
:10226000900037E090003FF07400900040F0786BF1
:10227000740126F640030221DA900040E0F40424C1
:1022800008F556E556D394054002C290E564D39410
:1022900001402FE54BD3946E4004D20E8002C20E53
:1022A000755605E564B40205A20EB34002800375BD
:1022B0005607E564B40306A20EB3B340028003756B
:1022C0005607E55765566008E55104F5528556579F
:1022D000E556B40708E5B54480F5B58006E5B55484
:1022E0007FF5B5E55664066005E556B40808E5B522
:1022F0004410F5B58006E5B554EFF5B575BB13E5AB
:1023000043B4050280030224137E017F00E5BE1260
:102310003F27E5BD2FFF50010E900000EEF0A3EF28
:10232000F07404123F198F46E563B4020280030281
:102330002410756B00756B00E56BD39403400302AA
:1023400023C7E56B900033123F3FE0D39546501A08
:10235000E56B900033123F3FE0F4042546FEE56B49
:1023600090002D123F3FEEF08017E56B9000331286
:102370003F3FE0C39546FEE56B90002D123F3FEED8
:10238000F0E56B6029E56B90002D123F3FFEE0FF0A
:10239000EE900031E0D39F4013E56B90002D123F8B
:1023A0003FE0900031F0E56B900032F0800E90003D
:1023B0002DE0900031F07400900032F0786B7401E1
:1023C00026F64003022338900082E07043E52A4558
:1023D000296036E558C39403500A900032E004C3E4
:1023E000940340028007900032E004F558E558D38A
:1023F0009402400A900032E004D394025002800715
:10240000900032E004F5588007900032E004F5585F
:1024100075BB180543D2ECE55ED394045003022447
:10242000FF75CF01C292AE35AF367488D39F741357
:102430009E4005A2A5B34014AE35AF367488D39F35
:1024400074139E4005A2A4B3400280487835120060
:102450003FAE35AF36EFB4883BEEB41337A2A5B329
:10246000500990004FE0D3955150028004055180EF
:1024700011A2A5B3500890004FE0655160028002A0
:10248000D207A2A4B35007E551D3940150028004AF
:102490001551C207A2A5B3B35006A2A4B3B340021C
:1024A0008006753600753500E55165526035E55199
:1024B00075F040A4FFAEF090032212001EE030E061
:1024C00003D38001C39293E55175F040A4FFAEF0B1
:1024D00090032312001EE030E003D38001C39294E6
:1024E000855152A20740057571CD80037571FFE5D6
:1024F00095C395714004C2878002D287022421A22D
:102500000DB3500DAE25AF2674E8C39F74039E40F3
:1025100002800575FFA0D20DAE25AF26EFD3942023
:10252000EE944E5003022613120481C28E758D0064
:10253000758B00754C00D28EC207757000756F00E8
:102540007571CD755104752400752300755400759F
:102550005A00C296900059E06004D2958002C2955C
:1025600090004AE0B40104D2978002C297900049DB
:10257000E0B40104D2A08002C2A0A209B34004D2F8
:10258000A28002C2A290006BE060181236E6A200A0
:10259000B34008E5B54408F5B58006E5B554F7F550
:1025A000B58002C20090006EE0601812383BA202B3
:1025B000B34008E5B54402F5B58006E5B554FDF530
:1025C000B58006E5B554FDF5B590000E74FDF0A399
:1025D00074E8F0E543B40603754300900025E4F089
:1025E000752600752500758D00758B00754C009063
:1025F0000024E0C394035008900024E004F0800617
:102600007403900024F0900024E0B40306E5B55470
:10261000FEF5B5AE27AF28EFD39410EE9427401CFB
:10262000C2CA75CD0075CC00752800752700D2CAC6
:0F263000754E00752A00752900755500020CC6FD
:1039ED0000000100013201640196019602000212ED
:1039FD0002240200020003000340038003C0040000
:103A0D000440048004C00500060006000600060000
:103A1D00060006000600060000FF01310163019556
:103A2D0001FF01FF0211022302FF02FF02FF033F0C
:103A3D00037F03BF03FF043F047F04BF04FF05FFA3
:103A4D0006FF06FF06FF06FF06FF06FF06FF06FF41
:103A5D000FAA0FA50F9F0F9A0F940F8D0F870F8031
:103A6D000F780F710F680F600F570F4E0F450F3BFB
:103A7D000F300F250F1A0F0E0F020EF50EE80EDB8D
:103A8D000ECC0EBE0EAE0E9F0E8E0E7D0E6C0E5A11
:103A9D000E470E340E200E0C0DF70DE20DCB0DB5AD
:103AAD000D9D0D850D6D0D540D3A0D200D050CE977
:103ABD000CCE0CB10C940C760C580C3A0C1B0BFB69
:103ACD000BDB0BBB0B9A0B790B570B350B130AF159
:103ADD000ACE0AAB0A870A640A400A1C09F809D4FF
:103AED0009B0098C09670943091F08FB08D608B2FC
:103AFD00088E086A0846082307FF07DC07B90796F2
:103B0D0007730751072F070D06EC06CA06AA06898B
:103B1D0006690649062A060A05EC05CD05B005928B
:103B2D0005750558053C0520050504EA04CF04B5C7
:103B3D00049C04820469045104390422040B03F427
:103B4D0003DE03C803B2039D038903750361034DAF
:103B5D00033B03280316030402F202E102D102C063
:103B6D0002B002A00291028202730265025702495D
:103B7D00023C022F02220216020901FD01F201E6AA
:103B8D0001DB01D001C601BB01B101A7019D01946B
:103B9D00018B0182017901700168016001580150AA
:103BAD000148014101390132012B0125011E011886
:103BBD000111010B010500FF00FA0FA60FA00F99CF
:103BCD000F920F8B0F840F7C0F740F6B0F620F58BA
:103BDD000F4E0F430F380F2C0F1F0F120F050EF73F
:103BED000EE80ED80EC80EB70EA50E930E800E6CF5
:103BFD000E580E420E2C0E150DFD0DE40DCB0DB114
:103C0D000D950D790D5D0D3F0D200D010CE10CC0D5
:103C1D000C9E0C7C0C590C350C100BEA0BC40B9E36
:103C2D000B760B4F0B260AFD0AD40AAA0A800A55F9
:103C3D000A2A09FF09D409A8097C0950092508F9A0
:103C4D0008CD08A10875084A081E07F307C8079D87
:103C5D0007730749072006F706CE06A6067E065708
:103C6D000630060A05E405BF059B057705540532A8
:103C7D00051004EF04CE04AE048F04710453043513
:103C8D00041903FD03E203C703AD0394037B036330
:103C9D00034B0334031E030802F302DE02CA02B60D
:103CAD0002A30291027F026D025C024C023C022CC7
:103CBD00021D020E020001F201E401D701CA01BE8C
:103CCD0001B101A6019A018F0185017A017001668A
:103CDD00015D0153014A01410139013101290121E0
:103CED0001190112010B010400FD00F700F000EABB
:103CFD0000E400DE00D900D300CE00C900C400BF2F
:103D0D0000BA00B500B100AD00A800A400A0009C51
:103D1D00009900950091008E008A00870084008133
:043D2D00007E007B99
:10266000751A00751900AE19AF1AAC17AD18EDC385
:102670009FEC9E401674FF123EF975CF01781A74D4
:102680000126F6500418E436F650DB22900786E463
:10269000F0A3F0751000750F00751300751400C2DB
:1026A0000FD21022C2AF75D900758F0375B7A5750B
:1026B000B7F190F800E4F0758F0175B7A575B7F123
:1026C000E50890F800F075B7A575B7F190F801E44A
:1026D000F075B7A575B7F190079DE090F802F07519
:1026E000B7A575B7F19007A1E090F803F075B7A50D
:1026F00075B7F190079EE090F804F075B7A575B72F
:10270000F190079FE090F805F075B7A575B7F190C7
:1027100007A0E090F806F075B7A575B7F19007A28D
:10272000E090F807F0758F0075D940D2AF2290077E
:1027300088E0B4AB61C2AF75D90075B62275F522D9
:10274000758F0375B7A575B7F1740090F600F07535
:102750008F01750A00750900AE09AF0A7413BE0037
:10276000279F402475B7A575B7F190078912001E01
:10277000E0FC90F60012001EECF0780A740126F6D8
:10278000500418E436F650D0758F0075F51175B603
:102790002075D940D2AF22C2AF75D90075F5227528
:1027A0000A00750900AE09AF0A7413BE00229F40EB
:1027B0001F90F60012001EE493FC90078912001E81
:1027C000ECF0780A740126F6500418E436F650D579
:1027D00075F51175D940D2AF22900788E0B4AA02EE
:1027E0008003022916C2AF75D90075B62275F5228D
:1027F000758F0375B7A575B7F1740090EE00F0758D
:10280000B7A575B7F1740090F000F075B7A575B76E
:10281000F1740090F200F075B7A575B7F1740090EF
:10282000F400F0758F01750A00750900AE09AF0A52
:1028300074FFC39F74019E402475B7A575B7F190CE
:10284000004E12001EE0FC90EE0012001EECF0782C
:102850000A740126F6500418E436F650CF750A00C3
:10286000750900AE09AF0A74FFC39F74019E40242E
:1028700075B7A575B7F190024E12001EE0FC90F0FE
:102880000012001EECF0780A740126F6500418E4D9
:1028900036F650CF750A00750900AE09AF0A74FF0D
:1028A000C39F74019E402475B7A575B7F190044E7F
:1028B00012001EE0FC90F20012001EECF0780A7488
:1028C0000126F6500418E436F650CF750A00750953
:1028D00000AE09AF0A74FFC39F74019E402475B710
:1028E000A575B7F190064E12001EE0FC90F40012A0
:1028F000001EECF0780A740126F6500418E436F64F
:1029000050CF758F0075F51175B62075D940D2AFCF
:10291000743A90074EF022900788E0B4AA02800330
:10292000022A54C2AF75D90075B62275F522758F8B
:102930000375B7A575B7F1740090E600F075B7A5FB
:1029400075B7F1740090E800F075B7A575B7F1742C
:102950000090EA00F075B7A575B7F1740090EC002F
:10296000F0758F01750A00750900AE09AF0A74FF92
:10297000C39F74019E402475B7A575B7F190004EB2
:1029800012001EE0FC90E60012001EECF0780A74C3
:102990000126F6500418E436F650CF750A00750982
:1029A00000AE09AF0A74FFC39F74019E402475B73F
:1029B000A575B7F190024E12001EE0FC90E80012DF
:1029C000001EECF0780A740126F6500418E436F67E
:1029D00050CF750A00750900AE09AF0A74FFC39F96
:1029E00074019E402475B7A575B7F190044E12008E
:1029F0001EE0FC90EA0012001EECF0780A7401263A
:102A0000F6500418E436F650CF750A00750900AE8A
:102A100009AF0A74FFC39F74019E402475B7A57562
:102A2000B7F190064E12001EE0FC90EC0012001E62
:102A3000ECF0780A740126F6500418E436F650CF0C
:102A4000758F0075F51175B62075D940D2AF743AFF
:102A500090074EF022900788E0B4AA028003022B70
:102A600092C2AF75D90075B62275F522758F0375C0
:102A7000B7A575B7F1740090DE00F075B7A575B70E
:102A8000F1740090E000F075B7A575B7F17400908F
:102A9000E200F075B7A575B7F1740090E400F07529
:102AA0008F01750A00750900AE09AF0A74FFC39F54
:102AB00074019E402475B7A575B7F190004E1200C1
:102AC0001EE0FC90DE0012001EECF0780A74012675
:102AD000F6500418E436F650CF750A00750900AEBA
:102AE00009AF0A74FFC39F74019E402475B7A57592
:102AF000B7F190024E12001EE0FC90E00012001EA2
:102B0000ECF0780A740126F6500418E436F650CF3B
:102B1000750A00750900AE09AF0A74FFC39F7401FE
:102B20009E402475B7A575B7F190044E12001EE0C3
:102B3000FC90E20012001EECF0780A740126F650B8
:102B40000418E436F650CF750A00750900AE09AFD7
:102B50000A74FFC39F74019E402475B7A575B7F131
:102B600090064E12001EE0FC90E40012001EECF0F5
:102B7000780A740126F6500418E436F650CF758FA3
:102B80000075F51175B62075D940D2AF743A90072B
:102B90004EF022900788E0B4AA028003022CD0C233
:102BA000AF75D90075B62275F522758F0375B7A577
:102BB00075B7F1740090D600F075B7A575B7F174CC
:102BC0000090D800F075B7A575B7F1740090DA00E1
:102BD000F075B7A575B7F1740090DC00F0758F0142
:102BE000750A00750900AE09AF0A74FFC39F74012E
:102BF0009E402475B7A575B7F190004E12001EE0F7
:102C0000FC90D60012001EECF0780A740126F650F3
:102C10000418E436F650CF750A00750900AE09AF06
:102C20000A74FFC39F74019E402475B7A575B7F160
:102C300090024E12001EE0FC90D80012001EECF034
:102C4000780A740126F6500418E436F650CF750A57
:102C500000750900AE09AF0A74FFC39F74019E405E
:102C60002475B7A575B7F190044E12001EE0FC90D4
:102C7000DA0012001EECF0780A740126F6500418EF
:102C8000E436F650CF750A00750900AE09AF0A7434
:102C9000FFC39F74019E402475B7A575B7F19006D8
:102CA0004E12001EE0FC90DC0012001EECF0780AD0
:102CB000740126F6500418E436F650CF758F00756F
:102CC000F51175B62075D940D2AF743A90074EF021
:102CD00022C2AF75D90075F522750A00750900AEDC
:102CE00009AF0A74FFC39F74019E401F90EE00124B
:102CF000001EE493FC90004E12001EECF0780A7463
:102D00000126F6500418E436F650D4750A00750909
:102D100000AE09AF0A74FFC39F74019E401F90F07C
:102D20000012001EE493FC90024E12001EECF0789C
:102D30000A740126F6500418E436F650D4750A00D9
:102D4000750900AE09AF0A74FFC39F74019E401F4E
:102D500090F20012001EE493FC90044E12001EEC50
:102D6000F0780A740126F6500418E436F650D4754B
:102D70000A00750900AE09AF0A74FFC39F74019E73
:102D8000401F90F40012001EE493FC90064E1200C7
:102D90001EECF0780A740126F6500418E436F6505A
:102DA000D475F51175D940D2AF22C2AF75D900756F
:102DB000F522750A00750900AE09AF0A74FFC39FBA
:102DC00074019E401F90E60012001EE493FC9000E8
:102DD0004E12001EECF0780A740126F6500418E436
:102DE00036F650D4750A00750900AE09AF0A74FFB3
:102DF000C39F74019E401F90E80012001EE493FCE4
:102E000090024E12001EECF0780A740126F650046F
:102E100018E436F650D4750A00750900AE09AF0AF9
:102E200074FFC39F74019E401F90EA0012001EE4CD
:102E300093FC90044E12001EECF0780A740126F602
:102E4000500418E436F650D4750A00750900AE092E
:102E5000AF0A74FFC39F74019E401F90EC001200E4
:102E60001EE493FC90064E12001EECF0780A7401EA
:102E700026F6500418E436F650D475F51175D9408D
:102E8000D2AF22C2AF75D90075F522750A00750957
:102E900000AE09AF0A74FFC39F74019E401F90DE0D
:102EA0000012001EE493FC90004E12001EECF0781D
:102EB0000A740126F6500418E436F650D4750A0058
:102EC000750900AE09AF0A74FFC39F74019E401FCD
:102ED00090E00012001EE493FC90024E12001EECE3
:102EE000F0780A740126F6500418E436F650D475CA
:102EF0000A00750900AE09AF0A74FFC39F74019EF2
:102F0000401F90E20012001EE493FC90044E120059
:102F10001EECF0780A740126F6500418E436F650D8
:102F2000D4750A00750900AE09AF0A74FFC39F7417
:102F3000019E401F90E40012001EE493FC90064E98
:102F400012001EECF0780A740126F6500418E436DC
:102F5000F650D475F51175D940D2AF22C2AF75D9EC
:102F60000075F522750A00750900AE09AF0A74FFF5
:102F7000C39F74019E401F90D60012001EE493FC74
:102F800090004E12001EECF0780A740126F65004F0
:102F900018E436F650D4750A00750900AE09AF0A78
:102FA00074FFC39F74019E401F90D80012001EE45E
:102FB00093FC90024E12001EECF0780A740126F683
:102FC000500418E436F650D4750A00750900AE09AD
:102FD000AF0A74FFC39F74019E401F90DA00120075
:102FE0001EE493FC90044E12001EECF0780A74016B
:102FF00026F6500418E436F650D4750A0075090018
:10300000AE09AF0A74FFC39F74019E401F90DC009D
:1030100012001EE493FC90064E12001EECF0780A9B
:10302000740126F6500418E436F650D475F511757F
:10303000D940D2AF22E51464046006E59964FF60CC
:10304000028031A20F4004D20F8027E5146008747B
:10305000E62514900023F0E513600874F025139022
:103060000023F0E514B4010280FE7514007513000E
:10307000C20F8002C20FE514903990F828287375AA
:103080001400E599B4FF03751301E599B4FE0375C7
:103090001302E599B4FD03751303E599B4FC0375B8
:1030A0001304E599B4FA03751305E599B4FB0675A5
:1030B0001401120481E599B4F9067514041204810F
:1030C000E599D394E54007E599C394F04002801652
:1030D0008599157514027E017F00E515C394E612EB
:1030E0003F278E0D8F0E900786E4F0A3F0E599D36D
:1030F00094C44007E599C394E64002802885991559
:1031000075140374E5C39515F50E750D00AE0DAF7E
:103110000E9039ED12002EE493F874019390078617
:10312000C8F0A3C8F0D2990235A4900786E0FEA3A8
:10313000E0FFEFC39400EE94054009EFD394FFEE57
:1031400094064013900786E0FEA3E0FF90004E1225
:10315000001EE599F0800385996C90078612000E99
:10316000900786E0FEA3E0FFEFB40106EEB407028D
:1031700080030233B490074EE0B43C028003023374
:10318000B4A20AB35005A20BB340030232A7C29CFB
:1031900090007AE090078CF0900057E090078DF057
:1031A000900062E090078EF0900063E090078FF04F
:1031B000900074E0900790F090007CE0900791F010
:1031C00090007DE0900792F0900080E0900793F0EF
:1031D000900081E0900794F090013AE0900795F01C
:1031E00090013BE0900796F090013CE0900797F04B
:1031F000900090E0900798F0900091E0900799F08F
:10320000900092E090079AF0900093E090079BF076
:10321000900094E090079CF0900095E090079DF05E
:10322000900096E090079EF0900097E090079FF046
:10323000900099E09007A0F090009AE09007A1F02C
:1032400090009BE09007A2F090009CE09007A3F014
:103250007400900082F01200C974AB900788F012DD
:0A326000272E74AA900788F0E558A5
:0639900002307F02312A23
:10326A009039B1F828287380121227D9800D1229B3
:0B327A00178008122A558003122B93C6
:0F39B10002327102327302327802327D023282A8
:10328500900788E4F090013AE0700C90013BE07003
:103295000690013CE060028004C20A8002D20A0264
:1032A50033A9C29C900078E0900789F090005EE019
:1032B50090078AF090005FE090078BF090007AE02D
:1032C50090078CF0900057E090078DF0900062E039
:1032D50090078EF0900063E090078FF0900074E007
:1032E500900790F090007CE0900791F090007DE0D1
:1032F500900792F0900080E0900793F0900081E0B5
:10330500900794F090013AE0900795F090013BE02A
:10331500900796F090013CE0900797F0900090E0C0
:10332500900798F0900091E0900799F0900092E056
:1033350090079AF0900093E090079BF0900094E03E
:1033450090079CF0900095E090079DF0900096E026
:1033550090079EF0900097E090079FF0900099E00D
:103365009007A0F090009AE09007A1F090009BE0F4
:103375009007A2F090009CE09007A3F074009000E5
:1033850082F074AB900788F012272E74AA900788F4
:10339500F01227D9122917122A55122B93D29C7590
:1033A50099FB80FED29C7514007513007599FB027C
:1033B50035A4900786E0FEA3E0FFEF4E70068599E1
:1033C50010750F00900786E0FEA3E0FF74016F4EB5
:1033D500701BAC0FAD10AA0DAB0EED2BFBEC3AFA42
:1033E5008A068B0790004E12001EE599F09007861D
:1033F50012000E900786E0FEA3E0FF74026F4E7088
:103405000C1200C98515997514007513000235A4B1
:10341500900786E0FEA3E0FF90004E12001EE5999E
:10342500F090078612000E900786E0FEA3E0FFAC41
:103435000DAD0E8F028E038C068D07903A25120076
:103445002EE493F9740193FEEAD39EEB9940098526
:1034550015997514007513000235A4900786E0FED2
:10346500A3E0FF90004E12001EE599F0900786122A
:10347500000E900786E0FEA3E0FFEFB40006EEB471
:10348500010280030235A490001CE0D394C7400BD1
:1034950090001CE0C394C8F516801A90001CE0D378
:1034A5009463400B90001CE0C39464F5168006906D
:1034B500001CE0F516E51675F002A4FFAEF08F6B63
:1034C500EF90004E123F3FEFFCE0FDEC90005112F3
:1034D5003F3FEDFCE0FDEC2DB5160280030235966D
:1034E5000FEF90004E123F3FE56BFFE0FCEF9000C1
:1034F50052123F3FECFFE0FCEFC39CB51602800380
:10350500023596E56B900050123F3FE56BFFE0FCFE
:10351500EF900053123F3FECFFE0FCEF2CB5167126
:10352500E56B900054123F3FE0C3951690079DF060
:10353500E56B900055123F3FE0C3951690079EF04E
:10354500E56B900058123F3FE0C3951690079FF03A
:10355500E56B900059123F3FE0C395169007A0F028
:10356500E56B90005A123F3FE0C395169007A1F016
:10357500E56B90005B123F3FE0C395169007A2F004
:103585001226A47599F975186475170012266080BE
:0F359500FE7599FF75186475170012266080FE89
:093996000233B70234150234605B
:1035A40022E51390399FF82828730236E5900786A0
:1035B400E0FEA3E0FF90001212001EE0F5999007D0
:1035C4008612000E900786E0FEA3E0FF74116F4E92
:1035D40070037513000236E58562990236E590079B
:1035E40086E0FEA3E0FF90004E12001EE0F599EF86
:1035F400B40107EEB4070375130090078612000E9A
:073604000236E5900787E0A4
:0F399F000235AE0235B10235DC0235E2023607E1
:10360B009039C0F82828738524990236DA852A99CF
:10361B000236DA8544990236DA8547990236DA851D
:10362B0051990236DA8560990236DA855699023657
:10363B00DA8558990236DA756E00900069E07006EB
:10364B00900068E060028016A2A44006E56E440478
:10365B00F56EA2A54006E56E4402F56E801A900049
:10366B004AE0B40106E56E4410F56E900049E0B4F3
:10367B000106E56E4420F56EA207B34006E56E44E5
:10368B0001F56EA209B34006E56E4408F56E856E32
:10369B0099803CA210B340077599FAC2108017A20B
:1036AB000CB3400575990F800B900023E0F59990B2
:1036BB000023E4F0C20C80178542998012854B9948
:0F36CB00800D85469980087599FC800375130062
:1039C00002361202361802361E02362402362A0247
:1039D000363002363602363C02364202369E023617
:0D39E000C30236C80236CD0236D20236D7F9
:0B36DA0090078612000E8003120048CB
:0339AE000236E2FC
:1036E5002290006BE0B4010385241190006BE0B4D7
:1036F5000203852A1190006BE0B403038544119001
:10370500006BE0B4040385471190006BE0B405033A
:1037150085511190006BE0B4060385561190006B3E
:10372500E0B4070385581190006CE0FE90006DE051
:10373500C39E50030237BC90006BE0D39404402C29
:1037450090006CE0D39511500990006DE0C3951180
:1037550050028002D20090006CE0D3951150099080
:10376500006DE0C395115002C200804990006BE0E6
:10377500B4041890006DE0C395115002D20090007A
:103785006CE0D395114002C200802A90006CE0C322
:103795009511500990006DE0D3951150028002D229
:1037A5000090006CE0D39511500990006DE0C39531
:1037B500115002C200807E90006BE0D39404402C2F
:1037C50090006CE0C39511400990006DE0D3951110
:1037D50040028002C20090006CE0C3951140099040
:1037E500006DE0D395114002D200804990006BE056
:1037F500B4041890006CE0C395115002C20090000B
:103805006DE0D395114002D200802A90006CE0C390
:103815009511400990006DE0D395114002D20090BA
:10382500006CE0D39511400990006DE0C3951140FF
:10383500028002C2002290006EE0B40103852411CB
:1038450090006EE0B40203852A1190006EE0B40387
:103855000385441190006EE0B40403854711900080
:103865006EE0B4050385511190006EE0B406038542
:10387500561190006EE0B4070385581190006FE073
:10388500FE900070E0C39E500302391190006EE077
:10389500D39404402C90006FE0D39511500990000B
:1038A50070E0C3951150028002D20290006FE0D300
:1038B50095115009900070E0C395115002C2028025
:1038C5004990006EE0B40418900070E0C395115063
:1038D50002D20290006FE0D395114002C202802A05
:1038E50090006FE0C395115009900070E0D39511D9
:1038F50050028002D20290006FE0D39511500990DA
:103905000070E0C395115002C202807E90006EE007
:10391500D39404402C90006FE0C3951140099000AA
:1039250070E0D3951140028002C20290006FE0C39F
:1039350095114009900070E0D395114002D20280A4
:103945004990006EE0B4041890006FE0C3951150E3
:1039550002C202900070E0D395114002D202802A83
:1039650090006FE0C395114009900070E0D3951168
:103975004002D20290006FE0D3951140099000708B
:0B398500E0C3951140028002C2022244
:093F3F002582F58250020583225F
:10002E00EF2F500205832582F582E5833E2EF58360
:01003E00229F
:08000300C3EF9DFFEE9CFE22FD
:08003F000806B60002180622B3
:0D000E00A3E004F07006123F35E004F0227C
:083F51000816B6FF0218162243
:0E3F1900048007C3CE13CECF13CFD5E0F6221F
:103D3100BC000FBE0008ED8FF084FFADF022E4FE61
:103D4100FF22BE000DEF60FE54F0606F20E703021A
:103D51003DE7EAC0E0EBC0E078017A0075F001EEE2
:103D610020E710EF25E0FFEE33FE0AC5F023C5F092
:103D710030E7F0EA5407F9096A7A007B006001082C
:103D8100C3EC9E40167004ED9F4010ED9FFDEC9E2C
:103D9100FCE5F0CA4ACA03F5F08005E5F003F5F049
:103DA100C3EE13FEEF13FFD9D77908CACBCAD8D017
:103DB100EAFEEBFFD0E0FBD0E0FA22EC8FF084FCCE
:103DC100ED54F045F0C48FF084FEEDC454F045F09D
:103DD100C48FF084FDEEC4FE54F02DFFEE540F3C71
:103DE100FEADF07C0022790078008FF0EC7E082097
:103DF100E70DC3CD33CD33C933C9C833C8DEF08431
:103E010049F9E5F08FF0BE00E6FD7C00E9FFE8FE30
:013E1100228E
:0E3F2700F88FF0A4FFE5F0CE88F0A42EFE2265
:103EF900600D782B023F03007830D8FED5E0F82218
:103F0900EEC0E07E00123D31EFFDEEFCD0E0FE2276
:03000B00023EA80A
:03001B00023EC3DF
:03002B00023EDEB4
:03000000023F4874
:093F480075817275D0000207FDBD
:0B001E00E5822FF582E5833EF583228A
:0A3F35000582D58202158315822251
:103EA800C0E0C0F0C083C082C0D075D0001207F255
:103EB800D0D0D082D083D0F0D0E032C0E0C0F0C003
:103EC80083C082C0D075D0001207F5D0D0D082D080
:103ED80083D0F0D0E032C0E0C0F0C083C082C0D050
:103EE80075D0001207F8D0D0D082D083D0F0D0E0BF
:013EF8003297
:00000001FF
